:10000000758107758920758841758DFD75985090AB
:1000100006471202C31202B912029B784074107B89
:10002000047600081470FA1204A6540F2440F876DF
:10003000551204A6540F2440F8E6B400F476571283
:1000400004A6540F2440F8E6B400F476501204A637
:10005000540F2440F8E6B400F476421204A6540F7C
:100060002440F8E6B400E6764212008E1201D61261
:1000700000C0120353B402031204781203B660E9FD
:100080009007B71202B91202C312029B808D791039
:100090007840E954037005740A120293747C1202CA
:1000A00093E6C39455B4000874551202930200B548
:1000B00074001202930819E970D8740A120293228C
:1000C0001202B91202B99004E51202C31202B91267
:1000D000029BB461071202D278FF8024B464071235
:1000E00002E978FF801AB4770712030278FF8010C4
:1000F000B4730712033178FF8006B4660312010758
:100100001202B9B8FFC922EB70111202B990077838
:100110001202C31202B9740178FF221B12038C90E1
:1001200005A11202C312029BB4640BE954039403A9
:10013000603012016622B46109E95403602412019F
:100140007922B4730EE9C313C313C394036013126B
:10015000018C22B4770CE9C313C313C360041201EA
:10016000A0221201C522E9042440F8E6C394577086
:10017000041201B4221201C522E9142440F8E6C396
:10018000945770041201B4221201C522E9240424F8
:1001900040F8E6C3945770041201B4221201C5223C
:1001A000E994042440F8E6C3945770041201B42281
:1001B0001201C5229005E11202B91202C31202B95E
:1001C00078FF7405229005D51202B91202C31202FB
:1001D000B978FF74012278407900C3E69455600431
:1001E000090880F6E95403600312022494036003B3
:1001F000120230E9C313C313C3600312023C940319
:10020000600312024912020922FF9007A51202C3DD
:10021000EB24301202939007AF1202C31202B912FC
:1002200002B9EF22FFE92440F818E6120256EF2245
:10023000FFE92440F808E6120256EF22FFE92440C5
:100240009404F8E6120256EF22FFE924402404F851
:10025000E6120256EF22603AE6B457061202A412E2
:1002600002B9B450061202AB1202B9B4420612022D
:10027000B21202B9B4510C1202A41202B91202ABAA
:100280001202B9B4430C1202A41202B91202B21241
:1002900002B922C299F5993099FD220E3098FCC21C
:1002A00098E599229004C11202C3229004D412024C
:1002B000C3229004B31202C322F5F0740A1202930F
:1002C000E5F022E493600AC299F5993099FDA38084
:1002D000F22212038CE95403700374012218E670B1
:1002E00041765508760074012212038CE954039478
:1002F00003700374012208E670287655187600749E
:10030000012212038CE9C313C313C37003740122C7
:10031000E89404F8E6700B7655E82404F876007447
:100320000122B44203740322B45003740222740401
:100330002212038CE9C313C313C394037003740123
:1003400022E82404F8E670DA7655E89404F876009A
:10035000740122B40106740012048F22B4020C90BE
:1003600005211202C31202B9740122B4030C9005D4
:100370004E1202C31202B9740222B4040C90057B1F
:100380001202C31202B9740122740122790078406A
:10039000C3E694556004090880F62279007840C3CA
:1003A000E694576010C3E69451600AC3E694436034
:1003B00004090880EA22600122FF1204A654030403
:1003C000C313C313C3B4002812039B1204A654071B
:1003D000C313C3B400051203F48015B4010512045D
:1003E00021800DB4020512044F800512043D8000E7
:1003F00060D6EF22E9607E14607B1460781460752B
:10040000142440F8E6B4000476578057B4550E9093
:1004100006041202B91202C37F0174012204F6809D
:1004200042E9941004604E04604B04604804604547
:1004300024102440F8E6B400D376578026E954030C
:100440006033E9142440F8E6B400C176578014E91B
:1004500054039403601FE9042440F8E6B400AD7629
:10046000578000E92440F8E6B4570576007401226D
:1004700014F674012274002212038CE92440F876E9
:10048000001204A6540F2440F8E670F5765522FFBA
:10049000EB9409600F1204A65407B405079007E116
:1004A0001202C30BEF22EEB400010475F0DDA424A8
:1004B00035FE22596F752068656172206261747320
:1004C00000596F7520736D656C6C20612077756DB8
:1004D00070757300596F75206665656C20612064C6
:1004E0007261667400506C6561736520707265732B
:1004F0007320772C612C732C6F72206420666F72CE
:10050000206120646972656374696F6E206F722068
:100510007072657373206620746F20666972652E31
:1005200000596F752066656C6C20696E746F206170
:10053000207069742E2020486176652061206E69E4
:1005400063652061667465726C6966652E00546827
:1005500065206261747320686176652063617272E0
:1005600069656420796F7520746F20612072616EF7
:10057000646F6D2073706163652100436F6E6772F5
:100580006174756C6174696F6E73212020596F7589
:100590002772652077756D70757320666F6F6421A3
:1005A00000506C656173652075736520772C612C34
:1005B000732C6F72206420746F2063686F6F736593
:1005C000206120646972656374696F6E206F6620B4
:1005D0006669726500596F75206D69737365642172
:1005E00000596F75206B696C6C65642074686520B8
:1005F00077756D7075732E2E2E6E69636520776F1B
:10060000726B21005468652077756D707573206674
:100610006F756E6420796F7521212020486F706599
:1006200020796F752772652066756C6C206F662067
:10063000766974616D696E7320616E64206D696E98
:100640006572616C73210057656C636F6D65207412
:100650006F2048756E74207468652057756D7075CD
:10066000732C20776865726520796F752068756EC8
:100670007420746865206D6F73742064616E6765A3
:10068000726F7573206F660A616E7920616E696D95
:10069000616C20746861742068617320657665728E
:1006A0002077616C6B656420746865206561727485
:1006B00068212020596F7572206F6E6C79206672E8
:1006C00069656E6420697320796F75722074727524
:1006D0007374790A626F7720616E64206172726F41
:1006E000772E2020496E20746865206361766573DB
:1006F000206172652070697473207468617420646D
:10070000726F7020796F7520746F20796F75722009
:10071000646561746820616E6420626174730A7438
:10072000686174207069636B20796F752075702023
:10073000616E64206D6F766520796F7520746F200F
:1007400072616E646F6D20706C616365732E202022
:10075000476F6F642048756E74696E67210A507226
:100760006573732061206B657920746F20636F6EF1
:1007700074696E7565210A00596F75206861766528
:10078000206E6F206172726F77732E2E2E626574E9
:100790007465722074727920746F2066696E6420AB
:1007A0006F6E652100596F752068617665200020A5
:1007B0006172726F777300506C656173652070723F
:1007C0006573732061206B657920746F20706C6194
:1007D0007920616E6F746865722067616D65210AAA
:1007E000000A0A596F7520666F756E6420616E206D
:0907F0006172726F77210A0A00A0
:00000001FF
